:020000020000FC
:10000000CECD00000000000020C0AFC194C00000B1
:1000100000009EC000000000000000000203040673
:10002000080C10182030406080000406080C1018DE
:100030002030406080A0C00000070F1F3F000D0D62
:1000400004050D050305030302004FB662FD0EC053
:10005000552009F00994C52DC095089483FDC795D6
:10006000C4BDC093A10064604FBE1895C0916400E8
:10007000089483FDC795C4BDC093A1006B7FC09158
:100080006400CF3F09F420C070FF02C082FD05C0AC
:100090004FBE939894989598189575FD0EC065FD80
:1000A0000CC0C091B300C0FD9298C1FDC298C2FDC2
:1000B000C198CAEFC095CA95F1F79398949895980E
:1000C0002092A1004FBE189524BCCC27C064C8BFA5
:1000D0006460F6CFC0CF70FFBECF65FDBCCF939AF2
:1000E000BACF70FFB8CF65FDB6CF949AB4CF70FF8A
:1000F000B2CF65FDB0CF959AAECF929A70FFABCFDD
:1001000065FDA9CFC7E0CA95F1F7939AA4CFC29A2B
:1001100070FFA1CF65FD9FCFC7E0CA95F1F7949A14
:100120009ACFC19A70FF97CF65FD95CFC7E0CA956A
:10013000F1F7959A90CF4FB6C9B7CF7EC9BF6E7F02
:10014000CCB5CE0DDDB5DF1DDBBDCABD4FBE1895EC
:100150003FB68F7EA9B7A072A2118061A9B7AF7D0B
:10016000A9BFA9B7AE7FA9BF7894A0916800AA23C0
:1001700041F085FD2BC0A0916800AA95A09368006E
:1001800025C040E050E085FD15C0A6B396FDA095C2
:10019000A0FD4FEFAEB5A06496FDAF7BAEBDAA2724
:1001A000A062A8BF8D7FA6B396FDA095A0FD5FEFCE
:1001B000451739F7A8E161FDA093680085FD03C0EC
:1001C000A8E1A093680040939700816085FD0EC070
:1001D000A0916900AA2331F0A0916900AA95A0938B
:1001E000690004C08061AA27A062A8BF80FF37C051
:1001F000A09197004A2F61FF8E7F85FD1CC0A091C2
:10020000B600A430C1F4403F08F040EFA42FA295FF
:10021000AF704A0F5091B800533069F0A695A6957B
:1002200050FD01C0A69552FD03C0A41B4A2F03C078
:100230004A0F08F44FEF40936100A72FA67079F0A2
:10024000A0916D00A695A69556E0A50F509161006E
:10025000A50FA093610018F4AFEFA0936100409147
:10026000B600443009F03EC0A0916100A093630045
:1002700040916300A0919C004A1708F04A2FA0917A
:100280009E004A1708F04A2F542EA091A200AA23DC
:1002900009F422C0542F5A1B10F4A42F50E0BA2E98
:1002A0008894AA1FAA2EA091A400A095AA22A50E08
:1002B00058F0A091A300A21509F0AA95AA0EA09348
:1002C000A30048F04A2D08C0A091A300BA1608F078
:1002D000A395A093A3004FEF409364007F7D485FF8
:1002E00008F07062A52DA03408F06860A09160004D
:1002F000A395A093600059F0F894A9B7A160A9BF95
:1003000084FF03C0A9B7A062A9BF3FBE1895A09102
:100310007400A395A093740041E0509168005523A8
:1003200029F085FF03C05A9550936800A09197006B
:10033000A13018F020929A000DC020929B002092CC
:10034000A500A0919A00AF5FA0939A0018F0AFEFBC
:10035000A0939A00F894A9B7A160A9BF84FF03C035
:10036000A9B7A062A9BF3FBE18953FB646B557B51D
:100370008F7EA9B7A072A2118061A9B7AF7DA9BF76
:10038000A9B7AE7FA9BF789481FD25C0AEB5AF7B7C
:1003900096FDA064AEBD8260A6B396FDA095A0FFB9
:1003A00005C0409365005093660041C1AEB5A0649E
:1003B00096FDAF7BAEBDAA27A062A8BF8D7F85FF4B
:1003C00001C028C140E0A6B396FDA095A0FD22C1C2
:1003D0004093970011C1AEB5A06496FDAF7BAEBD52
:1003E0008D7F61FF72C0AEB5AF7B96FDA064AEBDE0
:1003F000AA27A062A8BF8260409392005093930006
:10040000A09090004A19B09091005B09BB24A22CE7
:100410004C38520518F42092960049C0A091D6009D
:10042000AA2359F1483C520528F4A0E1BA2EAAE0CB
:10043000AA2E23C04836A1E05A0728F4A8E0BA2E15
:10044000AFE0AA2E1AC0403DA2E05A0728F4A4E06B
:10045000BA2EAEE1AA2E11C0403AA5E05A0728F400
:10046000A2E0BA2EACE3AA2E08C04839A8E05A0789
:1004700020F4A1E0BA2EA8E7AA2EC42EA0919400E1
:10048000CA1AD52EA0919500DA0ADD202AF4AFEF22
:10049000C094D094CA1ADA0A20929600A8E0A2105A
:1004A000A0E0CA14DA0618F4A1E0A09396004093E5
:1004B0009400509395004091920050919300409386
:1004C00090005093910002E097C0A09165004A1BF4
:1004D000A09166005A0B94FD82C093FD80C092FDEE
:1004E0007CC086FF03C0D52EC42E0CC05695479500
:1004F00091FD73C05695479590FD6FC0D52EC42EC3
:10050000D694C79461FD19C0AC2DAC51AD2DA2405D
:1005100008F005C0DD2089F4AC2DA85C70F4A09132
:100520006700A395AA2311F0A0936700AA3008F4EE
:1005300071C02092970081606DC0A0916700AA23CE
:1005400019F0AA95A0936700A22C5091BC0097FDCA
:1005500006C0A090CA00533011F4A090D200AAEFB8
:10056000AA0EA22DA21DCA18DA0A4FB74170533045
:1005700049F4442321F087FD05C0806803C087FF4C
:1005800001C08F77442359F0533031F4AFEFC0945A
:10059000D094CA1ADA0A03C040E050E020C05330B9
:1005A00049F4CC0CDD1CAAE0CA1AD20818F4A0E069
:1005B000CA2ED22CAFEFCA16D20418F04FEF50E07B
:1005C0000EC0A091AE00CA9E412D000C441F50E009
:1005D00008F012C04FEF50E00FC05695479594FFBA
:1005E00007C0552309F04FEFA42FA6954A0F521DBF
:1005F0004F3F520508F04FEF40939700816061FF35
:1006000009C0AFE1A095A923AB299A2F8F7DBB200C
:1006100009F48062A8E1A093680085FF03C0AAE006
:10062000A093680061FD03C085FD01C08F7E85FD3C
:1006300003C0A6E0A0936900F894A9B7A160A9BF80
:1006400084FF03C0A9B7A062A9BF3FBE189511E0FF
:100650000AC013E008C01AE006C01EE104C014E698
:1006600002C018EC00C005E1BB27BA95F1F70A9566
:10067000D9F71A95C1F708952AE338E709C020E3AE
:100680003CE806C02AE234EB03C025E238EC00C0A7
:1006900012E095FD9F7D95FF9062BB27C29ABA95A7
:1006A000F1F7949ABA95F1F79498BA95F1F7C29840
:1006B000BA95F1F7939AB091AF00BA95F1F7939884
:1006C000B7E8BA95F1F71A9521F7022FB22FBA952C
:1006D000F1F70A95D9F73A95D9F6C29A0895221BEF
:1006E00039E0001F3A9509F40895221F211B18F4E0
:1006F000210F8894F6CF0894F4CF622C722CB0E0CE
:100700008894B395221F331FE0F737952795889477
:10071000912E802E020B130B10F4192D082D10F4BE
:10072000889401C00894661C771CBA9571F7172D40
:10073000062D0895322D11232AF43A95009510952F
:10074000031B130BF894029F712C002D129F912C08
:10075000802C7894780C172D921C292DB4E06B2EE8
:100760002695179507956A94D9F7332321F00095BC
:100770001095031B130B08950091B6000430A1F1EE
:10078000B0919700B15008F010C0B0916100B093E3
:10079000630020927F0020928000209281002092AE
:1007A0008200209283006F7B1FC06090B60060645F
:1007B000B0916100B093620008E317EC20917A00D9
:1007C00030917B0036952795B62DBA9541F0369538
:1007D0002795B62DBA95BA9511F0369527958DDFE8
:1007E00000937F0010938000089500917F00B091E6
:1007F00062000B1B10918000120928F40038BFEF33
:100800001B0740F009C00F37120508F405C00FE7B9
:1008100010E002C000E81FEF0093840010938500F1
:10082000089500918400B09181000B0F1091850014
:10083000B09182001B1F20E03091850033230AF421
:100840002A95B09183002B1F1AF4203F40F00AC074
:100850002F3008F407C00FEF1FEF2FE003C000E0B8
:1008600010E020EF30916300B0919C003B1718F42A
:10087000323030F009C0B0918500BB235AF004C07B
:10088000B0918500BB2332F4009381001093820065
:100890002093830008952091D80000918400000FD8
:1008A00010918500111F46DF11232AF40038BFEF95
:1008B0001B0740F009C00F37120508F405C00FE709
:1008C00010E002C000E81FEF002352F0B091620078
:1008D000B01B0B2F18F0013008F00AC001E008C06F
:1008E00000950F5FB09162000B0F08F001C00FEF91
:1008F0000093860008952091D90000918200109104
:10090000830018DF11232AF40130BFEF1B0740F0EA
:1009100009C00F3F120508F405C00FEF10E002C038
:1009200001E01FEF112352F0B0918600B01B0B2F96
:1009300018F0013008F00AC001E008C000950F5F10
:10094000B09186000B0F08F001C00FEF0093630019
:1009500008950FEF677F71FD29C072FD09C06860BF
:10096000B0917B00BA3020F0B52DB03408F4677F29
:10097000B091D500BB23D1F0B0917B00BB23B1F087
:100980000FEF10917B00ABDEF894B091730072FD15
:10099000B5E00B9F112D002D7894112309F00FEF76
:1009A000B0919F000B1710F400919F0000939E00E0
:1009B000089500917A0010917B0000541140B0918D
:1009C0009E0010F4BA9501C0B39511F0B0939E004B
:1009D000089500C008952091B700B6B1B6FDFBCFD1
:1009E00004B115B1B6B1BF77B6B9B091AC00B3954B
:1009F000B093AC00B83060F12092AC00B091D4005C
:100A0000BB2321F1112329F0B091AD00BF3F61F06C
:100A100009C0B091AD000B1739F020F4BB2321F0D1
:100A2000BA9502C0B395E1F300919C00B093AD007C
:100A3000B93B50F400ECBA3A38F400E8BB3920F482
:100A400000E4BC3808F400E000939C00777F089530
:100A500010919C00B0E11B0F08F41FEF10939C0055
:100A6000B091B600B43081F000919C00B091630069
:100A7000B01B10F400916300B0919E000B1708F0BA
:100A80000B2F502E00936400B091AC00B73009F4E6
:100A90007860089502E3F894B091DA000B9F012D7D
:100AA000000C001F7894B0919C000B1710F000917F
:100AB0009C000093610000936300502E009364003B
:100AC00000939F00089520927A00B0EFB0937B00CE
:100AD0000895F8940CB51DB5209174007894309168
:100AE0007500609076000093750010937600031BEC
:100AF000160971FD03C076FD81C02BC07090770090
:100B0000209377002709222311F00FEF1FEF809029
:100B1000780090907900309378006092790069189D
:100B2000161910937C000091750010917600081939
:100B3000190920917A0030917B0036952795020F94
:100B4000131F10F40FEF1FEF00937A0010937B0038
:100B500029C020917A0030917B003901B4E08B2EBE
:100B6000B2E09B2E343010F08A949A94383010F012
:100B70008A949A94769467948A94E1F726193709AF
:100B8000992021F0169507959A94E1F7200F311FCF
:100B900020937A0030937B0028F43FEF30937A0063
:100BA00030937B00323008F4706471FF02C0B3E010
:100BB0000DC0B091C60000917100023838F0B395B5
:100BC000003A08F0B395B63008F0B5E09B2EB4E0DB
:100BD0008B2E10917B0000917A0024E016950795EA
:100BE0002A95E1F70819120928F0B02FB250B12F59
:100BF000B20910F402E010E0980126C020917A00BA
:100C000030917B003901769467946694669466947B
:100C10002619320906950695200F321D20937A0079
:100C200030937B00323008F07F7B04E036952795C7
:100C30003695279526952695201B10F0223008F42E
:100C400022E089019090C60060FDFECFE0908C000C
:100C5000F0908D006160B9B7B061B9BF380176FD21
:100C600044C07694679400938C0010938D00B92D46
:100C7000B330E1F0B0FD04C0060D171D930106C0AE
:100C8000000F111F0250120922E030E0B92DB330DD
:100C900068F020938E0030938F00009388001093AB
:100CA000890060928A0070928B003DC000938E0094
:100CB00010938F00209388003093890060928A00FF
:100CC00070928B0071FF10C0B0916D00B33060F076
:100CD00000918F0010917C001595010F28F022F0F3
:100CE00020928E0000938F001EC0669400938C00AB
:100CF000B92DB33091F0B0FD03C0060D262D03C011
:100D0000000F025022E0B92DB33038F020938E004E
:100D10000093880060928A0006C000938E002093A2
:100D2000880060928A0000917D0002FD035001302E
:100D300049F495FD12C0B0B7B860B0BFB0E0B06C78
:100D4000B7B90EC0023039F4B0B7B860B0BFB1E087
:100D5000B06CB7B905C095FDEECFB0B7B77FB0BFE7
:100D60000091A400000F10F4BBE60B270093A40031
:100D700060FDFECFB2E0B0936E006160B9B7B061C4
:100D8000B9BFB72FB670A1F020917A0030917B00E7
:100D900036952795F8940CB51DB5020F131F1BBD92
:100DA0000ABD6160B0E1B8BFB9B7B061B9BF7894AE
:100DB0000895606120927E0020E067FD20E206C079
:100DC000606120927E0020E267FD20E0789401E0DF
:100DD00076FD11C0B72FB67009F06F7EB0917B0021
:100DE000B55048F002E0B55020F003E0B55008F0EF
:100DF00006E071FD0AE060FD12C0B0917E00BB23E9
:100E000071F071FF08C0B0916D00B33020F0B09167
:100E10006E00BA9519F4789470615EC0AEDF789474
:100E200000000000F89476FD16C010917B0017308A
:100E300008F017E0B5E01B0F72FD10E183FF110F02
:100E400062FF110F71FD12E8B4B56090A100B619F0
:100E500090F2B10B80F2B0B71B2FB77FB0BFB8B123
:100E6000B0B713FDB860B0BFB0917E00B395B0933A
:100E70007E00B8B176FD06C0B1E071FDB2E0BA9572
:100E8000F1F7B8B1B072B21709F01BC071FF05C01D
:100E900003950A3008F00395AECF64FF97CF6F7EBD
:100EA0003CB56DB470907A0080907B00370D681C63
:100EB0006BBC3ABD6160B0E1B8BFB9B7B061B9BF52
:100EC00085CFB0916D00B23008F480CF64FD7ECF45
:100ED0000A9509F090CF7F7E20918E0030918F008F
:100EE000F894B0E1B8BF0CB51DB5020F131F1BBDC0
:100EF0000ABDE0908800F09089006160B9B7B061E8
:100F0000B9BF7894B72FB67039F0B0916D0072FF09
:100F1000B395B0936D0009C074FF07C067FD05C0AD
:100F200064FD03C0BF91BF91EEC4089500E063FF6C
:100F300003C064FF01C001E0F89410917100B7E0B4
:100F40001B9F212D102D7894200F269517952695FF
:100F500017952695179510937100183718F4B8E770
:100F6000B093710000917100B09172000B1720F0E6
:100F7000606293989498959860FDFECFE0908A0007
:100F8000F0908B006160B9B7B061B9BF0895AC98BB
:100F9000B2E095FD07C0F894B0937D00C29A929894
:100FA0007894EAC0F894B0937D00C29AC19878947E
:100FB000E3C0AC9AB3E082FF24C095FD11C002E00B
:100FC000F894B0937D00E7E8F0E00093B3009598C3
:100FD000C19A62FF02C0949A01C0C2987894CCC0B2
:100FE00002E0F894B0937D00E7E8F0E00093B300EE
:100FF0009398929A62FF02C0949A01C0C298789422
:10100000BBC095FD0BC0F894B0937D00E1E7F0E024
:10101000959862FF01C0949A7894AEC0F894B0930A
:101020007D00E1E7F0E0939862FF01C0949A789424
:10103000A3C0AC98B4E095FD07C0F894B0937D00D0
:10104000929AC198789498C0F894B0937D00C19A10
:101050009298789491C0AC9AB5E082FF24C095FD37
:1010600011C001E0F894B0937D00EDE7F0E000934B
:10107000B3009498C29A62FF02C0939A01C09298FA
:1010800078947AC004E0F894B0937D00E1E9F0E050
:101090000093B3009498C29A62FF02C0959A01C06F
:1010A000C198789469C095FD0BC0F894B0937D0009
:1010B000EBE6F0E0949862FF01C0939A78945CC0EC
:1010C000F894B0937D00E7E7F0E0949862FF01C0E8
:1010D000959A789451C0AC98B6E095FD07C0F89405
:1010E000B0937D00C19AC298789446C0F894B093AA
:1010F0007D00929AC29878943FC0AC9AB1E082FF8A
:1011000024C095FD11C004E0F894B0937D00E1E99E
:10111000F0E00093B3009398929A62FF02C0959A10
:1011200001C0C198789428C001E0F894B0937D0084
:10113000EDE7F0E00093B3009598C19A62FF02C01A
:10114000939A01C09298789417C095FD0BC0F894BB
:10115000B0937D00E7E7F0E0939862FF01C0959AB5
:1011600078940AC0F894B0937D00EBE6F0E095988F
:1011700062FF01C0939A78946F7D08952AE630E06B
:10118000F9012092B300939894989598929AC29AF4
:10119000C19A6B7F0895A4EBB0E009E00D9309E0DC
:1011A0000D9304E00D930FEF0D9303E00D930FEFFC
:1011B0000D930AE00D9303E00D9301E00D9301E020
:1011C0000D93A0ECB0E001E00D930FEF0D930D93A4
:1011D0000D930D930D9303E00D930FEF0D930FEF10
:1011E0000D930D9305E20D9300ED0D9308E20D9321
:1011F00000E50D9304E00D930FEF0D9302E00D93C6
:1012000000E00D930AE70D930FEF0D9300E00D93AF
:1012100001E00D9300E00D9303E00D9308952091FC
:10122000BB008B7F233009F48460B091BC00B330E5
:1012300019F09F7DB1FD90629F7BB091BD00B1FD23
:101240009064223011F0886001C0877F08950A956C
:10125000E00FF21DB4910895ECE1F0E00091B400CC
:10126000F6DFB093D800ECE1F0E00091B500EFDFDD
:10127000B093D900EAE2F0E00091BA00E8DFB09361
:10128000DA00B091D0000FEF1CE0B23011F400EAA8
:101290001AE0B33011F402E815E0009372001093E5
:1012A0007300E8E3F0E00091D700D1DFB093A20033
:1012B000089508952091CA003091CB00B091BC00F0
:1012C000B33009F43E5097FF02C020E03FEFB32F48
:1012D000B21B6B2EB25810F4B2E86B2E00E00395EF
:1012E000609EB12DBD57D8F30093AE00089590686D
:1012F000E1DFB3D920E030E0B0E16B2EAAD9B091A4
:1013000097002B0F321D6A94C9F7B4E036952795E4
:10131000BA95E1F7822E9F77CDDF0895F894E3E048
:10132000F0E0B9E0B7BFB491B078C1F3F894A895F4
:10133000B1B5B861B1BDB0E0B1BDB4E0BEBFBFE50D
:10134000BDBF1CDFB6E0B8BBB6E1B7BBB8E0B5BB0C
:10135000BCE1B4BBB4E0B2BBBCE3B1BB2224A0E0AF
:10136000B0E02D92AA31E9F7A0E6B0E00FEF2D92A0
:101370000A95E9F7B1E0B093A4000DDFF8D2B7E029
:10138000B06CB7B9B6B1B460B068B6B90091CC0072
:101390000093AF00B1E0B0936A00F89462D96CD9C1
:1013A0005CD96DD95AD96ED958D9F8940AEF1AEF89
:1013B000A6B396FDA095A0FF1FC01A95C9F70A9580
:1013C000B1F7E0E0FCE1B591B43E39F4B591B03E3F
:1013D00021F4B591BF3F09F40CC0E0E0F395F3951B
:1013E000B591B83F49F4B591B43931F4B591BA3AF1
:1013F00019F4EE27F695099412DF2EDF5ADF5ADF33
:101400000091CC000093AF00B9DEB2E0B3BFB2E010
:10141000BEBDB2E0B5BDB1E5B8BFB9BFB0B70B2F27
:10142000B77FB0BFB8B1B0B703FDB860B0BF0FD9D8
:101430007894CFDABEB5B06496FDBF7BBEBDB9B7B8
:10144000B062B9BFBB27B062B8BF8D7F0AD96260F6
:1014500033E02CE0B0919600BB2321F42CE03A95C8
:1014600009F4A3CFFAD880FFA0CF8E7FB091970068
:10147000B23078F3B92FBF710091990000939800B2
:10148000B0939900B01729F72A9521F76D7FBEB563
:10149000B06496FDBF7BBEBDBB27B062B8BF8D7F79
:1014A000B091D600BB2321F48062B92FB0709B2F7E
:1014B0008F7B20926700D3D885FF05C0B09167006D
:1014C000BA3008F08064C5D802E085FF01C000E0B2
:1014D000B0919700B017B8F3F894CED8CDD8CCD847
:1014E0007894BFD820928700B091BC00B33009F443
:1014F00074C0AFD8B091C000B13008F46EC0B091E4
:101500006A00B13008F469C085FD18C0B091970039
:10151000BF3F08F462C0F894B8D87894A0D8B091CE
:101520009700B130C0F7F894A7D895D8A5D878948B
:1015300096D8B0919700BF3FB0F3DAC2B3E09B2ECC
:101540009068F894B7DE78948AD8F8949F77B2DEE2
:1015500080909700B0919700BF37789408F445C009
:1015600076D8F89492D878949A9451F7C0DEB82D32
:10157000B550B093CB0075D8F89426D28CD278941D
:10158000BAE09B2E9068F89495DE789468D8F89429
:101590009F7790DE80909700B0919700BF37789446
:1015A00078F755D8F89468D856D866D878949A942D
:1015B00049F79DDEB82DBB5FB093CA0052D8F894AE
:1015C00003D278D278944BD8F89474DE7894B091A2
:1015D0009700BF3F08F498CF8BC200919700B0915D
:1015E00087000B1710F00093870039D801E0B09105
:1015F000BC00B35009F405E0B0919700B01708F0B3
:1016000073CFF89442D841D840D878942AD8209201
:101610006A0020926B0020926C00B0916B00B39531
:10162000B0936B00BF3F69F5B0916C00B395B09378
:101630006C00B091CE0009E1BA9559F002E3BA9579
:1016400041F00DE7BA9529F00AEFBA9511F0209212
:101650006C00B0916C00B017A0F0B0916C00BA951E
:10166000B0936C00B4EBB0936B00B091CD00B0932D
:10167000AF00F8940AD87894B091CC00B093AF0042
:10168000EED7E9D7B0916800BB2319F485FF01C0FC
:101690008CCE01E085FD01C006E0B0919700B01747
:1016A00008F4BBCFB091BC00B35009F0D8D7B091CB
:1016B0006800BB2309F479CEF89460DD20926100C4
:1016C0002092620020926300522C209264002092AB
:1016D000A3007894B091B900BB0FB093A000209202
:1016E0007F00209280002092810020928200209230
:1016F00083002092AC0060E070E020927100B8E0BE
:10170000B093AC007860A3D7B7E073FDB6E0B06CDF
:10171000B7B9B6B1B068B064B6B9B6B1B6FDFDCF71
:1017200004B115B1B6B1BF77B6B9112309F00FEF07
:101730000093AD0050D9B8E0B093AC0078608090D1
:10174000BB00B2E0B093BB006ADD8092BB00F894AE
:10175000BFEFB0939C009ED9B0916100B0939C0004
:10176000B0939D00B0939E007894B1E0B093610077
:10177000B09363005B2EB0936400B093A600B09169
:101780009B00B093A500B091BC00B33019F49F7DCD
:1017900087FD90627160726020926D009CDCADDC10
:1017A00092D997D990D995D98ED906C0F89437DDBA
:1017B00078942092AC00777F03DBDED7B7DBE7DBE2
:1017C00088D9F7DA66FD11D876FFC3D876FDF1D84F
:1017D000ADDBEFDB7ED9F4DA66FD23D8A7DB29DCAD
:1017E00078D9E7DA66FD57D8A1DB35DC72D9E8DABB
:1017F00066FD81D89BDB6FDC6CD9DBDAB7E073FD6B
:10180000B6E0B06CB7B9B6B1B068B064B6B98EDB4B
:1018100074DC5FD9E0D871FF26C067FD24C0B091A9
:101820009F00B0939C00B0939D00B0919B00B0933B
:10183000A500B1E0B093A60018E12CE0B0916D00D6
:10184000B11758F07D7F746020936F00B0919F00B6
:10185000B0939C00B0939E0006C0B0919700B13049
:1018600008F0AACF5AC072FF10C067FD0EC0B09139
:101870006F00BA9511F47B7F99CFB0936F00B09150
:101880009700B13008F098CF48C020927000B09116
:101890009A000AEFB01708F040C085FF04C0B0916D
:1018A0006800BB23D1F1B091BC00B33081F495FD49
:1018B00003C087FD04C00BC087FF01C008C067FDDF
:1018C00006C06068B0919F00B0939C008ACF00EF83
:1018D00067FF05C0B0919F00B0939C0000E2B091FB
:1018E0007B00B01708F468CF67FF17C06F779F7D44
:1018F00087FD90627460B2E1B0936F00B0919F0079
:10190000B0939C0059CFB0917000B395B093700024
:10191000B0919700BB2309F002C020927000F894A8
:101920002DDC8090BB00B2E0B093BB0078DC8092ED
:10193000BB00209261002092620020926300522C32
:10194000209264002092A0007E7F789480D616DCDE
:10195000B7E0B06CB7B9B6B1B460B068B6B985FFDE
:1019600005C0B0917000B53008F01FCD52CEEDE04B
:10197000F0E023D0053509F01BC0EEE0F0E01DD00B
:101980000A3A09F015C03AE0A4EBB0E0E3E0F0E079
:1019900014D00D9331963A95D9F738E1A0ECB0E028
:1019A000EFE0F0E00AD00D9331963A95D9F702C0F6
:1019B000F2DB0AD0E7E2F0E00895E199FECFEEBB5A
:1019C000FFBBE09A0DB308951ED03AE0A4EBB0E05F
:1019D000E3E0F0E00D910FD031963A95D9F738E178
:1019E000A0ECB0E0EFE0F0E00D9105D031963A9533
:1019F000D9F712D00895E199FECF0DBBEEBBFFBB26
:101A0000E29AE19A0895EDE0F0E00FEFF4DFEEE006
:101A1000F0E00FEFF0DF0895EDE0F0E005E5EBDF3B
:101A2000EEE0F0E00AEAE7DF08953091B0000091BF
:101A3000B100313011F40093B400323011F400934E
:101A4000B500333011F40093B600343011F4009334
:101A5000B800353011F40093BA00363011F4009319
:101A6000C600373011F40093BB00383011F40093F6
:101A7000D700393011F40093D0003A3011F40093BC
:101A8000BC003B3011F40093BD00089525E0E9D57A
:101A90002A95E9F70895F0D5F2D5F4D5F6D5DBD53A
:101AA000EBD5EDD5EFD5F1D5D6D5E6D5E8D5EAD548
:101AB000ECD50895EAD5E6D5E2D5DED5CCD5E5D589
:101AC000E1D5DDD5D9D5C7D5E0D5DCD5D8D5D4D5A8
:101AD00008958090B0009090B100CED5CDD5CCD5F2
:101AE000BAD58A94D1F7D1D5B6D59A94E1F70895AD
:101AF000F894D1DF7894CADFC9DFB1E0B093B000C9
:101B0000B1E0B093B1002092B200F894E2DF789493
:101B1000B5E06B2E70909700A4D5B09197007B161E
:101B2000C9F7B13018F0BF3F40F107C07EDFF8942D
:101B30004BDFB1DFB8E0B1BDA9DF6A9459F7B091CE
:101B4000B200B395B093B200B33008F4DECF9EDF9D
:101B5000B091B100B395B093B100F894B091B000DA
:101B6000BA95EEE3F0E0EB0FF21D04917894039543
:101B7000B091B100B01708F4C6CF88DF87DFB0910D
:101B8000B000B395B093B000B091B000BC3008F491
:101B9000B7CF01DBF89418DFB8E0B1BD77DFBECB7B
:00000001FF
